:1000000000308A00702900000A108A100A11820745
:1000100028340C34013406340A108A100A1182077D
:10002000413468346F346A3400341E308400000870
:100030000319292801308D008C018C0B1D288D0B94
:100040001C284A308C008C0B232800000000800BF9
:100050001A2800340608C339A500240D8C008C0D25
:10006000FC308C050C083C392504860006148316E8
:100070000610000083120610831606108312003447
:10008000A208031D4528861046288614831686106C
:100090008312A30E2308A4002A20A30E2308A40081
:1000A0002A200D308C008C0B5328003414309E0015
:1000B0001520C3308316860583128610831686109A
:1000C000831206108316061083129B011B08023C44
:1000D000031C722802309E0015200330A4002A2041
:1000E0009B0A66280D308C008C0B74280230A4000B
:1000F0002A200D308C008C0B7B289B011B08023CB6
:10010000031C8E281B0804209C00A2011C08A300CD
:10011000402002309E0015209B0A7E287429013061
:100120001E02A0001F08023C031D98284030A007B3
:1001300020088038A100A2012108A300402000343B
:100140001D088C000C300C020319B3280A300C0275
:100150000319BB280D300C020319C12808300C020A
:100160000319C628CB28A2010130A3004020023089
:100170009E001520D72801309E0002309F008F205E
:10018000D72801309E009F008F20D728A201103071
:10019000A3004020D7281D081F3C031CD12807308E
:1001A0009D050130A2001D08A3004020D72800347F
:1001B0009E0104309D009D080319EC2883168515C7
:1001C0008312851DE52804309D0029308C008C0B9E
:1001D000E72800009D03DB28831685158312851907
:1001E000F6280A308C008C0BF328EC28D0308C00D9
:1001F0008C0BF8281B0884008316851500308312A9
:100200008519013080009D011D08033C031C222933
:10021000A6308C008C0B0A29000003109E0C83165C
:1002200085158312851D162908309E071F181A2967
:1002300005121B29051683160512013083129F062D
:100240009D0A04291C0884001E08800001308D00CE
:1002500000341E088D011D02031831291D088C0071
:100260003D298C0108309F009D0D8C0D1E080C024D
:1002700003188C008D0D9F0B342900340D081B08CA
:100280009D0064309E0029210C089B000D08303031
:10029000031D51291C189C159C1957291C1A203024
:1002A00053299C111C128D070D089D00A0201B08CE
:1002B0009D000A309E0029210C089B000D0830305B
:1002C000031D66299C196A291C1A20308D070D0808
:1002D0009D00A02030309B071B089D00A02000340B
:1002E00084011F308305562805309E0015209B0190
:1002F0001B080C209B0A9D00A02004301B02031D3C
:10030000782903309C002E309D00A0209C0B83296F
:1003100002309B0096309E0015209B0B8A298E018F
:100320008F019001910192019301940195011A307E
:100330009B0016309C00D8208D08031DA02997290A
:100340009A080319A42997291A309B0016309C009B
:10035000D8208D08031DAD2997291A309B0017302E
:100360009C00D8208D08031DB62997291A309B00C0
:1003700018309C00D8208D08031DBF299729170825
:1003800016070F3918020319C729920A9729013055
:100390001602FD3E0318D829033E702A17088E0066
:1003A000900AD82917088F00910AD829950AD829C8
:1003B00001309E009F008F2058309D00A0200E0825
:1003C0009B0011309C003E2120309D00A020100891
:1003D0009B0010309C003E2112089B0010309C00B6
:1003E0003E2113089B0010309C003E2120309D00D0
:1003F000A02020309D00A02001309E0002309F00F0
:100400008F2059309D00A0200F089B0011309C00C8
:100410003E2120309D00A02011089B0010309C0040
:100420003E2114089B0010309C003E2117089B00C1
:1004300010309C003E2120309D00A02020309D00E7
:10044000A020831605108312051401309E0015208C
:100450000E08970017089703003A0319392A153038
:100460008C008C0B312A00009708031D382A0030BD
:100470002A2A83160510831205108316851083120D
:10048000851401309E0015200F0897001708970368
:10049000003A0319552A15308C008C0B4D2A0000A8
:1004A0009708031D542A0030462A831685108312AC
:1004B00085100E081E3C8D000F080D0297001708CE
:1004C0009703003A03196E2A15308C008C0B662AAC
:1004D00000009708031D6D2A00305F2A97296300EA
:0E04E0000A108A140A118207CE29D229D629C1
:02400E00F13F80
:00000001FF
